:1000000025007F0A08072A00080500080F0C0600D3
:100010008605A605010CA60702090509860405093F
:10002000110AA60400080F0C06008604A60505099F
:100030000509010CA60702098605040C86070209BA
:100040000008A305C50AA305D70A080C2F006E00F7
:100050006E0303070E0403060E052109E9060E05CB
:10006000EF02280AC90523090008080C2F00C9045B
:10007000ED06C90523096D0303070D0403060D05ED
:10008000EF02370AFF06480A2109030CE9060209B4
:10009000000811022D000609350910022D0035094E
:1000A0000C022D0035091309A40B11022D000609BD
:1000B000350910022D003509060911022D000D0524
:1000C0003509250913090E022B008A0BA3051A0A0C
:1000D0000008A3053B0AA3054C0AA305680AA3056B
:1000E0006F0A7700780079000008A305760AA30557
:1000F0007D0AA00C3100BA021A02300000081F0C61
:1001000002003F0C06007F0071097709030C99007B
:100110004307850A7A00830B7F001F06970A6A004F
:10012000010C2900AC0C28006F096B099F0A6A00BA
:100130006900180C2800DF0768006F096B09A30528
:10014000000A060C3700100C2400060900022D00DE
:100150003509A402F702A60A13096F09800C2800CA
:10016000160C2900000C2A006B093E024306BF0A48
:10017000D00C3B00160C3C00000C3D008D0A0B021D
:100180003700510C97000307CC0A800C3B00160C7B
:100190003C00000C3D008D0A730074007500040CD7
:1001A00032001F07D90ADF07D90A180CB700030766
:1001B000B80A37024306DF0A6609F702DC0AA6041A
:1001C000FF056D003509000CBF07140C2D00350923
:1001D000150243060A0C2D0092032D013509130266
:1001E00043060A0C2D0034024307F80A0A0C3400B7
:1001F00094032D0135096D00DF07FF0A0E0C2D0059
:100200003509FF04BF06230B9F065F0B5F065F0BDC
:100210001F06190B71097709040C99004306AD0AF2
:100220000607250B2607420B3F0446060B0B1F054E
:100230008D0A71097709040C99004306AD0A460737
:100240001A0B1F048D0AA305A60A3F06380B710975
:1002500077090606330B2607700B020C990003077B
:10026000280B3F05380B770006070A0BF703340B02
:100270006F096A006900010C280069096D093F06D1
:1002800075098D0A3F06550B710977092606500B33
:100290000607810B020C99000307450B3F05550B20
:1002A000770026070A0BF703510B6F096A006900F4
:1002B000010C28006B096D093F0675098D0A71094B
:1002C00075096606720B4606680B5F049F040A0BED
:1002D000F703610BF803610B2607AB0B9F06AD0B11
:1002E0005F05380B790075094606790B5F049F049A
:1002F0000A0BB9023F0C99004307730B9F06AD0B25
:10030000380BA3058A0A1B0C2400020C3600FA00E5
:100310007909550A0B022000A402F602880B7D0021
:10032000DF04FC06DF05FC04BF04DC078D0AA3051F
:10033000830ADF06FC051B0C2400020C3600FA00C1
:10034000790900022C00490A7509A402F602A00BE3
:10035000BF04FC048D0AFF0C3A009F05BA02140C7E
:080360009A004307830BAB0B6D
:100400000B0233000C0234000D023500720075033C
:10041000020C7501A00C35017403030615051404C4
:100420007303030614051305C40C3000030C3100DC
:10043000A304A10A050CF3010A0C93000307230A85
:100440000A0CB300B402020CF4010A0C9400030776
:100450002C0A0A0CB400B5020A0C95000307330AF3
:100460000A0CB500B2020A0C92000307390A0A0C02
:10047000B200A304680A0802EB010306460A090257
:10048000EC0103064A0A0A02ED01390AEC033F0AAD
:10049000AD023F0AED03430A7E000802AB000307EA
:1004A0005F0A0902AC0003075A0A0A02AD000307FB
:1004B000BE02390A010CAD000307BE02550A010C49
:1004C000AC000306670A010CAD000307BE02510A27
:1004D0000B023B000C023C000D023D00390A1B02DE
:1004E0002B001C022C001D022D00390A7700780019
:1004F000F703780AF803780A390AF703820AF8033F
:10050000820AB902390A7D00160C3C00BC0C3B0083
:10051000A3048C0A770026069A0A06078A0AF703BC
:100520008B0ADF07950ADF04960ADF052607960A7D
:10053000A3048D0A720075007400760077007800BD
:10054000790016023300BF05A304DF0A1602D601A4
:100550003A00F703AE0AF803AE0AB9020606C10A6A
:10056000040C99004306C30A2606A60A770026074C
:10057000B60AF703B70AB6020A0C960043079E0AAA
:100580009A0AA304830BA304990B1F0C060086058B
:10059000E904A605010CA606D00A08072A000805EA
:1005A0008606E905D30AD40AD50AA604390A0F0C2F
:1005B0000600C907E50A8605DD0A0000020C86066A
:1005C000E90A08072A000805E90A8604E70AE80A92
:1005D000E90AA605010CA606F00A08072A00080584
:0A05E000F10AF20AF30AA604390A30
:00000001FF
